:020000040000FA
:030000000200916A
:030003000224E7ED
:030023000221CEE9
:03002B000224FBB1
:03003B000223E9B4
:06003E0053D9BF79012235
:1000440000000080FB12003EB9000302008BE49024
:1000540001A1785379088002F0A3D8FCD9FA90085A
:10006400F3AA82AB839000A0783079028015E493E0
:10007400A3AC82AD838A828B83F0A3AA82AB838CE8
:0D008400828D83D8E9D9E712257D12004452
:0F00910075D0007581BF7510A17511010200496E
:1000A000506C6561736520707265737320616E7941
:1000B000206B657920746F20636F6E74696E75654F
:1000C0002E2E2E203F007C205452494720523130A2
:1000D000302052313030207C203530306E732F6428
:1000E0006976207C2035562F646976207C3F007C21
:1000F0002053796E63207C20496E74207C20436FEE
:10010000725A20434841207C20436F725A20434852
:1001100042207C3F00523130303F0053796E633FC4
:100120000000025980013530306E733F312E30753A
:10013000733F322E3075733F332E3075733F342E3C
:100140003075733F352E3075733F31302075733FF6
:1001500031352075733F32302075733F3430207550
:10016000733F35302075733F36302075733F37301D
:100170002075733F38302075733F39302075733FD9
:1001800031303075733F31323075733F31343075F3
:10019000733F31353075733F31363075733F3138C9
:1001A0003075733F32303075733F33303075733F85
:1001B00034303075733F35303075733F312E306DCC
:0F01C000733F322E306D733F342E306D733F011D
:1001CF00C3E498F8E499F91202108026C3E49AFA6E
:1001DF00E49BFBE920E7E9120210E498F8E499F9AF
:1001EF0022C3E498F8E499F9120210E498F8E4991C
:1001FF00F9C3E49AFAE49BFB22EB20E7CFE920E76F
:10020F00E0B90010BB0008E88AF084F8AAF022E4F5
:10021F00FBC8FA22EB70227B10C833C8C933C9332D
:10022F005007C39AC3DBF280069A50012ADBEAC853
:10023F0033F4C8C933F4C9FA2275F008E4C833C8D7
:10024F00C933C933C99AC99B5004C92AC93BD5F0D0
:10025F00ECFBC833F4C8E4C9FA22600D08C6A2E764
:10026F0013C618C613C6D5E0F322700422600D180A
:10027F00C6C333C608C633C6D5E0F41822251010FE
:10028F00AF08F510400215118008F5104002151146
:10029F00D2AF22C0D0251010AF08F51050020511B3
:1002AF008008F51050020511D2AFD0D0222510F5DD
:1002BF0082E43511F583222510C582C0E0E51134A3
:1002CF00FFC583C0E0E510C3958224F9F8E4C5A803
:1002DF00858311858210C5A8E8CEF0A3E520F0A391
:1002EF007808E608F0A3DEFAEFF0A3E58124FBF827
:1002FF00E608F0A3E608F0A30808E608F0A3E6086E
:10030F00F0A315811581D0E0FED0E0F8158115819D
:10031F00E8C0E0EEC0E022851183851082E0A3FEE5
:10032F00E0A3F5207808E0A3F608DFFAE0A3FFE0EA
:10033F00A3C0E0E0A3C0E0E0A3C0E0E0A3C0E0E41E
:10034F00C5A8858210858311C5A8D083D08222D0FD
:10035F0083D082C5F0E493A3C5F0C395F0F5F0E424
:10036F0093A3C395F04005E5F0048001E475F00216
:10037F00A42582F582E5F03583F583E493A3C0E0ED
:0C038F00E493C0E022D083D082E9C0E0FB
:10039B00E493A3C386F0C5F095F0F908E493A38624
:1003AB00F0C5F095F0700BE493A3C3994005E904F5
:1003BB008002A3E475F002A42582F582E5F0358373
:1003CB00F583D0E0F9E493A3C0E0E493C0E022D03E
:1003DB0083D082CCC0E0E493A360061204041470B3
:1003EB00FAE493A360061204231470FAD0E0FCE441
:1003FB0093A3C0E0E493C0E022C0E0E493A3D39CBA
:10040B005010E493A3C39C400AD0E0D0E0D0E002AC
:10041B0003F7A3A3A3D0E022C0E0E493A36C70097D
:0E042B00D0E0D0E0D0E00203F7A3A3D0E0229F
:1004390000402060105030700848286818583878F3
:1004490004442464145434740C4C2C6C1C5C3C7CA3
:1004590002422262125232720A4A2A6A1A5A3A7AB3
:1004690006462666165636760E4E2E6E1E5E3E7E63
:1004790001412161115131710949296919593979A3
:1004890005452565155535750D4D2D6D1D5D3D7D53
:1004990003432363135333730B4B2B6B1B5B3B7B63
:1004A90007472767175737770F4F2F6F1F5F3F7F13
:1004B9000040206010503070084828681858387873
:1004C90004442464145434740C4C2C6C1C5C3C7C23
:1004D90002422262125232720A4A2A6A1A5A3A7A33
:1004E90006462666165636760E4E2E6E1E5E3E7EE3
:1004F9000141216111513171094929691959397923
:1005090005452565155535750D4D2D6D1D5D3D7DD2
:1005190003432363135333730B4B2B6B1B5B3B7BE2
:1005290007472767175737770F4F2F6F1F5F3F7F92
:1005390000000000000000000000000000000000B2
:1005490000000060000000000000007000000000D2
:100559003000007C000000003F80007E00000000A9
:100569003FF8007F8000000001F8007FE0000000F4
:100579000108003FF80000000100000FFE00000024
:1005890001000003FF80000021000000FFF00000CF
:100599003F0000001FFC00183FF8000007FF80180B
:1005A90007F8000000FFE01800180000003FFC18E1
:1005B900000000000007FF9C007800000000FFFC1D
:1005C9003FF8000000003FFC3FF8000000001FFC5E
:1005D900180000000001FFFC06000000000FFFFCEE
:1005E9000180000000FFFFFC00E0000007FFFFFCA6
:1005F90007F800007FFFFFE03FF80003FFFFFE0060
:100609003F00001FFFFFF0000C00007FFFFF00000C
:100619000300007FFFF0000000C0007FFF800000A2
:0E0629000038007FFC0000000008003FFC00CD
:1006370000003000000FFF80000030200001FFE0C5
:100647000000107000003FFC00000020000007FFC2
:1006570080000000000001FFF00000000000003FE4
:10066700FC0000000000000FFF80000000000001F8
:10067700FFE00000007000007FF80000007C000031
:100687001FF83000007F000007FC3F80007FE0007C
:1006970001FC0F80003FFC00007C0100003FFF00D1
:1006A700003C0180003FFFE0001C0180003FFFF895
:1006B700000008000038FFFF00183F0000383FFF28
:1006C700E0183F80003807FFFC182280003801FF40
:1006D700FF9822800038003FFFF813800078003F22
:1006E700FFFC030000780039FFFC000000780038A9
:1006F7003FFC01800078003807FC3F800078003815
:1007070001FC3F8000780038003C3000007C003856
:10071700001C0C00007E0038001C0600003F00385B
:10072700001C0180001FC038001C0080000FE0384B
:10073700001C00000003E018001C00000000E0009F
:10074700001C000000000000001C0000000000006A
:100757000E1C0000006000000FFC3C00007C000045
:100767000FFC3C70007F000007FC3C78007FE00036
:1007770001FC2178007FF800007C2108007FFF0042
:10078700000C2108003FFFE000003F080007FFF8CA
:1007970000183FF80001FFFF00181EF800003FFF98
:1007A700E0180078000007FFFC1C0000000001FFB4
:1007B700FF9C30000000003FFFFC300000000007F6
:1007C700FFFC300000000001FFFC0000007000008B
:1007D7003FFC0000007C000007FC0400007F0000D5
:1007E70001FC0600007FE000003C0500007FF800E8
:1007F70000000480003FFF0000000460003FFFE0AE
:1008070000003E30003FFFF800183FF80038FFFFB8
:10081700001807F800383FFFE0180438003807FFD2
:0C082700FC1C0000007801FFFF9C00009A
:100833000078003FFFFC000000780007FFFC000089
:1008430000780001FFFC0000007800003FFC00007E
:100853000078000007FC00000078000001FC0000A5
:1008630000780000003C0000007C00000000000055
:10087300007E000000000000003F80000000000038
:10088300001FE00000000000000FE0000000000077
:100893000003E000000000000000E0000000000092
:1008A3000000000000000000000000000000000045
:1008B3000000000000000000000000000000000035
:1008C3000000000000000000000000000000000025
:1008D3000000000000000000000000000000000015
:1008E3000000000000000000000000000000000005
:1008F300000000000000000000780000000000007D
:10090300007F00000000000000FFC00000000000A6
:1009130000FFE0000000000000FFE00000003000E6
:1009230000F8E00000003FC000F0000000003FF8C6
:1009330000E00000000001F800E0000000000118E2
:1009430000E00007F800011800E0000FFE000118A6
:1009530000E0001FFF00001800F0003FFFC0000090
:100963000070003FFFE000780078007FFFE03FF871
:10097300007C00FFC7F03FF8003C01FF81F818003E
:10098300003F01FF00780600001FC7FE003C018006
:10099300000FFFFC003C00E0000FFFFC001C07F809
:1009A3000007FFF8001E3FF80001FFF0000E3F00B4
:1009B3000000FFE0000E0C0000003FC0000E03002B
:1009C30000000700001E00C0000000000C1E0038DD
:1009D300000000000FFE0008000030000FFE300092
:1009E3000007FFC00FFE3020000FFFF003FC107064
:1009F300001FFFFE00FC0020003FFFFF0018000067
:100A0300007FFFFFC0000000007FFFFFE000000049
:100A130000FF83FFF800000000FE003FFC00000021
:0C0A230000F80007FE00000000F00001D9
:100A2F00FF00300000F000007F803F8000E00000FA
:100A3F001FC00F8000E000000FC0010000E00000A9
:100A4F0007E0018000E0000003F0018000F00000EB
:100A5F0001F008000070000000F83F000070000077
:100A6F0000783F8000780000003C228000380000B2
:100A7F00003C2280003C0000001C1380001C000082
:100A8F00001E0300001E0000000E0000000F0000FB
:100A9F00000E0180000F0000000E3F8000070000D5
:100AAF00000E3F8000030000000E30000000000029
:100ABF00001E0C0000000000001E060000000000D9
:100ACF00003E01800001FC00187E0080000FFFC077
:100ADF001FFE0000001FFFF01FFC0000003FFFFE85
:100AEF001FFC0000007FFFFF83FC0000007FFFFF63
:100AFF00C0F8000000FFFFFFF000000000FE03FF42
:100B0F00F800000000F8003FFC00000000F00007B4
:100B1F00FF00002000F00001FF803E2000E00000F9
:100B2F007FC03FE000E000001FC00FF800E00000B2
:100B3F0007E0003800E0000003F0000000F00000C4
:100B4F0001F000000070000000F8000000780000C5
:100B5F000078300000780000003C3000003C0000BE
:100B6F00003C3000003E0000001C0000001F000091
:100B7F00001E3800001F8000000E3C00000FE00038
:100B8F00000E3C780007F000000E22780003FC00F6
:100B9F00000E22080001FF00001E21080000FFC008
:100BAF00001E210800007FF8003E20F800003FFFE4
:100BBF0080FE00F800001FFFFFFE0078000007FF17
:100BCF00FFFC0000000001FFFFFC3C000000007F65
:100BDF00FFF83FF00060001FFFF03FF8007C0003BC
:100BEF00FFE020F8007F00003F002088007FE0003A
:100BFF0000002088007FF80000003C88007FFF0085
:100C0F0000003FB8003FFFE000001FB80007FFF8EB
:0C0C1F00001800380001FFFF0018000062
:100C2B0000003FFFE0180000000007FFFC18000069
:100C3B00000001FFFF9800000000007FFFF800009C
:100C4B0000000077FFF8000000000071FFFC0000BF
:100C5B00000000703FFC00000000007007FC00006B
:100C6B000000007801FC000000000078003C000050
:100C7B0000000038001C00000000003C001C0000BD
:100C8B000000003E001C00000000003F001C0000A4
:100C9B000000001F801C00000000001FC03C000073
:100CAB000000000FF07C000000000007FFFC0000BC
:100CBB0000000003FFFC000000700003FFFC0000BD
:100CCB00007C0000FFF80000007F00007FF80000B0
:100CDB00007FE0001FF00000003FFC0007E0000079
:100CEB00003FFF0000000000003FFFE0000000009D
:100CFB00003FFFF8000000000038FFFF0018000065
:100D0B0000383FFFE0180000003807FFFC18000018
:100D1B00003801FFFF9800000038003FFFF800008B
:100D2B000078003FFFFC000000780039FFFC00005A
:100D3B00007800383FFC00000078003807FC00000A
:100D4B000078003801FC000000780038003C0000FF
:100D5B00007C0038001C0000007E0038001C0000E6
:100D6B00003F0038001C0000001FC038001C0000B2
:100D7B00000FE038001C00000003E018001C00000E
:100D8B000000E000001C000000000000001C000040
:100D9B00000000000E1C0000000000000FFC000013
:100DAB00000000000FFC00000000000007FC00002A
:100DBB000000000001FC000000000000007C0000AF
:100DCB0000000000000C000000000000000000000C
:100DDB000000000000000000000000000000000008
:100DEB000070000000000000007000000000000018
:100DFB000078000000000000007C000000000000F4
:100E0B00007C000000000000007E000000000000DD
:0C0E1B00007E007800000000007F00FC5A
:100E270000000000007F80FE00000000007FC0FE81
:100E370000000000007FC0FF00000000007DE0FF11
:100E470000000000007DF00780000000007CF80330
:100E570080000000007CF80180000000007C7C011D
:100E6700C0000000007C3E01C0000000007C1F8322
:100E7700C0000000007C1FC3C0000000007C0FFF03
:100E8700C0000000001807FFC0000000000003FFBB
:100E9700C0000000000001FFC0000000000000FFCC
:100EA7008000000000F8003F8000000000FC000008
:100EB7000000000000FE00000000000000FE00002F
:100EC7000000000000FE000000000000007E00009F
:100ED70000000000003E00000000000000000000CD
:100EE70000000000000000000000000000000000FB
:100EF70000000000000000000000000000000000EB
:100F0700000000000000000000000000001FF000CB
:100F170000000000003FFE0000000000007FFF000F
:100F270000000000007FFFC00000000000FFFFE09E
:100F37000000000000FFFFF80000000000FC1FF8A1
:100F47000000000000F003FC0000000000F000FEBD
:100F57000000000000E0003F0000000000E0001F6C
:100F67000000000000F0000F8000000000F0000704
:100F77008000000000780003C0000000007C000330
:100F8700C0000000003E0001C0000000003F00015B
:100F9700C0000000001FC003C0000000000FF007E2
:100FA700C00000000007FF1FC00000000003FFFF94
:100FB700C00000000001FFFFC00000000000FFFFAD
:100FC7008000000000003FFF8000000000000FFFCE
:100FD70000000000000001FC00000000000000000D
:020FE700000008
:100FE90000000000000000000000000000000000F8
:100FF900000000000000FF33FF3300000000000084
:1010090000000700070000000000070007000000BB
:101019002001FE1FFE1F20012001FE1FFE1F2001CF
:1010290038063C0E6408FF3FFF3F84091C0F180770
:101039001E30331C1E07C00170001C1E0733011E21
:101049001E1FB331E120E120B3311E1F001B803187
:101059000000000000000B00070000000000000075
:1010690000000000F807FF3F0738000000000000FB
:101079000000000000000000000000000000000067
:101089000000000000000000000000000000000057
:101099000000000000000000000000000000000047
:1010A9000000000000000000000000000000000037
:1010B9000000000000000000000000000000000027
:1010C90000000000000000300030000000000000B7
:1010D9000030003C000FC003F0003C000F0003008B
:1010E900FC0FFE1F0336812161201B30FE1FFC0F00
:1010F900042004200620FF3FFF3F0020002000209D
:101109000C380E3C032601238121C3207E203C207C
:10111900061803304120412041204120E330BE1F01
:10112900000FE00FFC081F08833F803F00080008FC
:101139003F0C3F1C2130212021206130C11F810F2C
:10114900E00FF81F5C3046204320C130811F010F9A
:10115900010001000100013C813FF1037F000F0004
:101169001C0FBE1FE33041204120E330BE1F1C0F7E
:101179003C207E20C32081308118830EFE07FC01AC
:101189000000000000000000000000000000000056
:101199000000000000000000000000000000000046
:1011A9000000000000000000000000000000000036
:1011B900200120012001200120012001200120011E
:1011C9000000000000000000000000000000000016
:0C11D9000000000000000000000000000A
:1011E50000000000000000000000000000000000FA
:1011F50000000000FC3FFE3F030101010101030166
:10120500FE3FFC3FFF3FFF3F412041204120E330AF
:10121500BE1F1C0FFC0FFE1F0330012001200330F1
:101225000E1C0C0CFF3FFF3F012001200120073859
:10123500FE1FF807FF3FFF3F41204120412041208D
:1012450041200120FF3FFF3F810081008100810097
:1012550081000100FC0FFE1F033001208120833037
:101265008E1F8C0FFF3FFF3F4000400040004000B5
:10127500FF3FFF3F012001200120FF3FFF3F0120ED
:1012850001200120000C001C00300020002000304F
:10129500FF1FFF0FFF3FFF3FC000E00138071C0E97
:1012A5000F3C0330FF3FFF3F0020002000200020BF
:1012B50000200020FF3FFF3F7800C003C0037800F7
:1012C500FF3FFF3FFF3FFF3F1C007000C0010007CD
:1012D500FF3FFF3F0000000000000000000000008D
:1012E50000000000FF3FFF3F810081008100C30037
:1012F5007E003C000000000000000000000000002F
:1013050000000000FF3FFF3F810081008101C31FF6
:101315007E3E3C203C0C7E1C6330E120C1218331A4
:101325008E1F0C0F030003000300FF3FFF3F030068
:1013350003000300FF0FFF1F0030002000200030D6
:10134500FF1FFF0F3F00FF01C00F003C003CC00F17
:10135500FF013F00FF01FF3F003EC001C001003E0D
:10136500FF3FFF010000000000000000000000003A
:101375000000000000000000000000000000000068
:10138500000000000138013E8127C121612039207C
:101395001F200720000000000000000000000000E2
:1013A5000000000000000000000000000000000038
:1013B5000000000000000000000000000000000028
:1013C5000000000000000000000000000000000018
:0C13D5000000000000000000000000000C
:1013E10000000000000000000000000000000000FC
:1013F1000000000000000000001E403F20212021CD
:1014010020212011E03FC03FFF3FFF3F401020203F
:1014110020206030C01F800F800FC01F603020204F
:101421002020202060304010800FC01F603020201D
:1014310020204010FF3FFF3F800FC01F603220225D
:1014410020226022C033801320002000FE3FFF3F96
:1014510021002100230002008007C00F6018201026
:1014610020104008E03FE03F0000000000000000C5
:101471000000000000000000000020202020E33FC9
:10148100E33F0020002000000000000000000000F9
:101491000000000000000000FC3FFC3F00060007C8
:1014A100800DC01860302020000001200120FF3F86
:1014B100FF3F002000200000E03FE03F6000C01F30
:1014C100C01F6000E03FC03FE03FE03F4000200020
:1014D10020006000C03F803F800FC01F603020208F
:1014E10020206030C01F800FE03FE03F4004200813
:1014F1002008600CC007800300000000000000000D
:101501000000000000000000E03FE03FC00040009C
:101511006000600060004000C010E0312021202305
:1015210020262024603C4018000020002000FE1FDF
:10153100FE3F202020200000E01FE03F002000208F
:1015410000200010E03FE03FF003F007001C0030F6
:101551000030001CF007F003000000000000000054
:10156100000000000000000000000000000000007A
:101571000000000000000000E001E0270026003824
:101581000018000EE007E00120302038202C202632
:101591002023A021E02060200000000000000000C6
:1015A1000000000000000000000000000000FF3FFC
:1015B100FF3F0000000000000000000000000000EC
:1015C100000000000000000000000000000000001A
:0C15D1000000000000000000000000000E
:1015DD0000000000000000000000000000000000FE
:1015ED0000000000000000000000000000000000EE
:1015FD0000000000000000000000000000010203D8
:10160D000405060708090A0B0C0D0E0F1011121315
:10161D001415161718191A1B1C1D1E1F2021222305
:10162D002425262728292A2B2C2D2E2F30313233F5
:10163D003435363738393A3B3C3D3E3F40414243E5
:10164D004445464748494A4B4C4D4E4F50515253D5
:10165D005455565758595A5B5C5D5E5F000000004B
:10166D00000000000000000000000000000000006D
:10167D00000000000000000000000000000000005D
:10168D00000000000000000000000000000000004D
:10169D00000000000000000000000000000000003D
:1016AD00000000000000000000000000000000002D
:1016BD00000000000000000000000000000000001D
:1016CD00000000000000000000000000000000000D
:0C16DD0000000000000000000000000001
:1016E900FFFF0000020004000600080012001C00B1
:1016F90026004E00620076008A009E00B200C600F5
:10170900EE0016012A013E0166018E0156021E03F2
:08171900E603020004000800D1
:1017210075B9807A14001AEA70FB43B9C0E5B9E5CE
:10173100B9A2E550FA75A90275B28322C082C083AD
:1017410012172175A40D75A5E775A70175D40F753D
:10175100D50775DF0175E10575E242438805E58826
:1017610075E401D2A8C2AA759810758D0D538EF437
:10177100E58E438E08858D8B53890FE5894389203A
:10178100D28E7401900978F0D2ACD28C438922E5D3
:1017910089438E0CE58E758CB075C18043E6017569
:1017A100D80053D9BF75D90275DA4275DB4275FC91
:1017B1000775EA07D2DE75C80475CA0175CB01C287
:1017C100ADC283D282D280C292D291D290D2B0C223
:0817D10096D296D2AF0221C9A5
:1017D900D296D282D29275A6FFD291C291D291D2DB
:1017E90083C29275A083C280D280D29275A002C2B0
:1017F90080D280C283D283C29275A085C280D280F2
:10180900D29275A003C280D280C283D283C292755C
:10181900A08CC280D280D29275A093C280D280C29D
:1018290083D283C29275A091C280D280D29275A0D0
:1018390001C280D280C283D283C29275A083C28042
:10184900D280D29275A000C280D280C283D283C2D4
:101859009275A03EC280D280D29275A0B0C280D2C9
:1018690080C283D283C29275A03FC280D280D292B5
:1018790075A003C280D280C283D283C29275A04070
:10188900C280D280D29275A010C280D280C283D287
:1018990083C29275A041C280D280D29275A056C2ED
:1018A90080D280C283D283C29275A042C280D28084
:1018B900D29275A013C280D280C283D283C292759C
:1018C900A043C280D280D29275A046C280D280C283
:1018D90083D283C29275A044C280D280D29275A06D
:1018E90023C280D280C283D283C29275A045C280AE
:1018F900D280D29275A076C280D280C283D283C2AE
:101909009275A046C280D280D29275A000C280D2C0
:1019190080C283D283C29275A047C280D280D292FC
:1019290075A05EC280D280C283D283C29275A0485C
:10193900C280D280D29275A04FC280D280C283D297
:1019490083C29275A049C280D280D29275A040C24A
:1019590080D280C283D283C29275A017C280D280FE
:10196900D29275A061C280D280C283D283C292759D
:10197900A02BC280D280D29275A0F9C280D280C237
:1019890083D283C29275A01BC280D280D29275A0E5
:1019990014C280D280C283D283C29275A01AC28037
:1019A900D280D29275A011C280D280C283D283C262
:1019B9009275A01CC280D280D29275A00DC280D22D
:0319C90080C28356
:1019CC00D283C29275A01FC280D280D29275A03DE4
:1019DC00C280D280C283D283C29275A019C280D237
:1019EC0080D29275A00AC280D280C283D283C29266
:1019FC0075A019C280D280D29275A01AC280D280F2
:101A0C00C283D283C29275A019C280D280D2927541
:101A1C00A012C280D280C283D283C29275A01EC291
:101A2C0080D280D29275A020C280D280C283D28311
:101A3C00C29275A03CC280D280D29275A060C28046
:101A4C00D280C283D283C29275A03DC280D280D292
:101A5C009275A040C280D280C283D283C29275A0FC
:101A6C0034C280D280D29275A038C280D280C28318
:101A7C00D283C29275A035C280D280D29275A03822
:101A8C00C280D280C283D283C29275A024C280D27B
:101A9C0080D29275A038C280D280C283D283C29287
:101AAC0075A024C280D280D29275A03CC280D28014
:101ABC00C283D283C29275A016C280D280D2927594
:101ACC00A01CC280D280C283D283C29275A001C2F4
:101ADC0080D280D29275A006C280D280C283D2837B
:101AEC00C29275A055C280D280D29275A000C280DD
:101AFC00D280C283D283C29275A002C280D280D21D
:101B0C009275A000C280D280C283D283C29275A08B
:101B1C0003C280D280D29275A000C280D280C283D0
:101B2C00D283C29275A004C280D280D29275A000DA
:101B3C00C280D280C283D283C29275A005C280D2E9
:101B4C0080D29275A0EFC280D280C283D283C2921F
:101B5C0075A006C280D280D29275A000C280D280BD
:101B6C00C283D283C29275A007C280D280D29275F2
:101B7C00A000C280D280C283D283C29275A008C258
:101B8C0080D280D29275A001C280D280C283D283CF
:101B9C00C29275A009C280D280D29275A08FC280E9
:101BAC00D280C283D283C29275A022C280D280D24C
:0D1BBC0092C28375A60075A0FF2275A6FFDA
:101BC900D283C29275A003C280D280D29289A0C268
:101BD90080D280C283D283C29275A006C280D2808D
:101BE900D292EBF5A0C280D280C283D283C2927511
:101BF900A007C280D280D292EAF5A0C280D280C268
:101C090083D283C29275A022C280D280D292C2832B
:101C19002274F81202C6EAFEEBFFD29675A6FF7A85
:101C2900007B007900121BC6D283C29275A022C222
:101C390080D280D292C2837AF97BC0EFFCD2838CA6
:101C4900A0C280D280EEF5A0C280D280C283D283A6
:101C59008CA0C280D280F5A0C280D280C283EA1A49
:101C690070DBEB1B70D77F0102032674F41202C6E6
:101C7900890BEC24E9F582E43415F583E4939001AA
:101C8900E2F0F508750900740378081202799001E9
:101C9900E0E508F0A3E509F08A088B099001E0E086
:101CA900F8A3E0F9E8C333F8E933F9E824E9FEE9F0
:101CB900340FFF750A08AA08AB09A90B121BC678CD
:101CC900007920D283C29275A022C280D280D2929A
:101CD900C283750C0E8E828F83E49358FAA3E49322
:101CE90059FBEA7001EB60059001E380039001E57F
:101CF900E0FCA3E0D283F5A0C280D280ECF5A0C2BB
:101D090080D280C283E9C313F9E813F8150CE50CF6
:101D190070C3EE24020E0EEF3400FFE5082401F52E
:101D290008E5093400F509150AE50A70897F0502F5
:101D3900032674F11202C6890AECFEED8A0C8B0D9A
:101D4900750839750905750E56750F01F50BAA0C3D
:101D5900AB0DA90A121BC6D283C29275A022C280FA
:101D6900D280D292C2838508828509837B087C80D0
:101D79007A08E4935CD283600C850BA0C280D28080
:101D8900EEF5A0800A75A074C280D28075A053C2F6
:101D990080D280C283ECC313FC1AEA70D5A31BEB73
:021DA90070CCFC
:101DAB00E5082408F508E5093400F509E50C2401DC
:101DBB00F50CE50D3400F50DE50E24FFF50EE50FE2
:101DCB0034FFF50FE50E7002E50F70807F080203FC
:101DDB002674F81202C69001E5E4F0A3F09001E737
:101DEB007460F0A374FCF09001E374FFF0A3F09027
:101DFB0001E5E0FAA3E0FB121C1A9001DCE0D2E053
:101E0B00F07C8F7D017A017B007912121EF57C8F9D
:101E1B007D017A017B0079DF121EF57E007F007554
:101E2B0082197583098019EEFAEFFBEA75F00AA4A3
:101E3B00FAADF075F00AEBA42DFB7901121C74A31B
:101E4B00E0FAEE24010EEF3400FFEAFC743F6A70F7
:101E5B00D67E007F007582427583098019EEFAEFFA
:101E6B00FBEA75F00AA4FAADF075F00AEBA42DFBB2
:101E7B0079E1121C74A3E0FAEE24010EEF3400FF9B
:101E8B00EAFC743F6A70D69001E374E6F0A374FF2A
:101E9B00F07582687583097E507F008012EEFAEF31
:101EAB00FB7901121C74EE240AFEEF3400FFA3E051
:101EBB00FAFC743F6A70E69001E374BFF0A3741DE3
:101ECB00F07582687583097E827F008012EEFAEFCF
:101EDB00FB7901121C74EE240AFEEF3400FFA3E021
:101EEB00FAFC743F6A70E6021C6F74F61202C68924
:101EFB000A8A088B09ECFEEDFF121BC69001DCE091
:101F0B00A2E0E492E012035E0001861F1B1F471F35
:101F1B009001E7E0FAA3E0D283F5A0C280D280EA79
:101F2B00F5A0C280D280C283EEF8EFF974FF281EB1
:101F3B0074FF39FFE87001E970D6803F9001E7E04C
:101F4B00FAA3E0D283F5A0C280D280EAF5A0C280CA
:101F5B00D280C283AA08AB09A90A121BC6E50824C2
:101F6B0001F508E5093400F509EEF8EFF974FF28DF
:101F7B001E74FF39FFE87001E970C17F030203266D
:101F8B0074F71202C69001E774EFF0A3747BF0753F
:091F9B0008197509007E147F008D
:101FA400AA08AB09EEF9121BC69001E7E0FAA3E018
:101FB400D283F5A0C280D280EAF5A0C280D280C2CA
:101FC40083EE2405FEEF3400FFC3EE94E0EF9400AB
:101FD40040CEE5082419F508E5093400F509C3E500
:101FE40008948FE509940140B37508147509007EBF
:101FF400007F00EEFAEFFBA908121BC69001E7E090
:10200400FAA3E0D283F5A0C280D280EAF5A0C28010
:10201400D280C283EE2405FEEF3400FFC3EE948F1A
:10202400EF940140CEE5082419F508E5093400F5DC
:1020340009C3E50894E0E509940040B39001DCE0AD
:10204400C2E0F07CC87D007AC87B007914121EF5CA
:10205400E0D2E0F07C8F7D017A007B007978121E5B
:10206400F59001E7E4F0A3F07C8F7D01FAFBF9120F
:072074001EF57F02020326A6
:10207B00C082C08374019001CFF09001DDE0441267
:10208B00F012216A900976E09001BBF09001CFE04D
:10209B009001BCF09001D0E09001BDF09001D1E037
:1020AB009001BEF074029001CFF09001DDE044127C
:1020BB00F012216A9001CFE09001BFF09001D0E0C7
:1020CB009001C0F09001D1E09001C1F07408900133
:1020DB00CFF09001DDE04412F012216A9001CFE0C5
:1020EB009001C2F09001D0E09001C3F09001D1E0DB
:1020FB009001C4F0740E9001CFF09001DDE0C2E1CD
:10210B00F0D2E4F012216A9001CFE09001C5F0907B
:10211B0001D0E09001C6F074379001CFF09001DD53
:10212B00E0C2E1F0D2E4F012216A9001CFE090011D
:10213B00C7F09001D0E09001C8F0740D9001CFF082
:10214B009001DDE0C2E1F0D2E4F012216A9001CF00
:10215B00E09001C9F09001D0E09001CAF0805FC01F
:10216B0082C0839001DDA2A8E092E3F0C2A8D2E086
:10217B00F0A2E45007C2E4F0D2E28002C2E2F0D255
:10218B00C5E0A2E040FB9001DFE0A2E25028E0A214
:10219B00E14023E49001D0F09001D1F07401900163
:1021AB00CFF09001DDE0C2E2F0D2C5A2E040FC909E
:1021BB0001DFE0C2E2F09001DDE0A2E392A8D08360
:1021CB00D08222C0E0C0D0E8C0E0E9C0E0EAC0E0C5
:1021DB00C082C083A29840030223779001DDE0A266
:1021EB00E050169001B8E0FA74012AF0EAC3941596
:1021FB00400C9001DDE0C2E0F0E49001B8F09001FA
:10220B00B1E070079001B4E4F0A3F0C298E59990A7
:10221B0001BAF09001B1E0C394114003022377900F
:10222B0001BAE0C0E09001B4E024A1F8A3E03401CE
:10223B00F988828983D0E0F09001B1E004F090013D
:10224B00B4E02401F0A3E03400F09001B1E064109D
:10225B0060030223779001B0E0640D600302235FFB
:10226B009001DBC0829001A1E0A2E0758301D082D6
:10227B00E092E3F09001DBC0829001A2E0A2E07556
:10228B008301D082E092E1F09001DBC0829001A348
:10229B00E0A2E0758301D082E092E2F09001DBE0F6
:1022AB00A2E1400DE0A2E240089001A4E09001D52C
:1022BB00F09001A5E09001D0F09001A6E09001D143
:1022CB00F09001A7E09001CFF09001A8E090097683
:1022DB00F09001A9E0900977F09001AAE09001B984
:1022EB00F09001DBC0829001ABE0A2E0758301D0DE
:1022FB0082E092E6F09001B9E064017004C2B08014
:10230B0002D2B09001DBE0A2E3E05014E0C2969061
:10231B0001D3E4F0A3F0D2969001DBE0C2E0800C95
:10232B00A2E140F7E0A2E240F2E0D2E0F09001CF70
:10233B00E0640170089001DDE0D2E18010E06402FE
:10234B0060F3E0640860EE9001DDE0C2E1F0E49040
:10235B0001B18017E49001B1F09001DBE0D2E0F025
:10236B00E0C2E3F0E0C2E1F0E0C2E2F0A299505625
:10237B00C299900974E07002A3E0603A900974E08E
:10238B00F8A3E0F99001B2E0687003A3E06970076D
:10239B009001B6E4F0A3F09001BAE0F5999001B684
:1023AB00E02401F0A3E03400F0900974E024FFF086
:1023BB00A3E034FF800F9001B2E0F8A3E0F990099D
:1023CB0074E8F0A3E9F0D083D082D0E0FAD0E0F942
:1023DB00D0E0F88004D083D082D0D0D0E032C0E0FF
:1023EB00C0D0C082C083C0F0A2C250030224E074EC
:1023FB00F055C01203DA000380A524C02B24E00E95
:10240B0024E024900976E0C333F5C253C2FE900159
:10241B00DDE0A2E4E492E045C2F5C2C2C50224E0CD
:10242B00A2C1506D9001DDE0A2E450030224E0A2B2
:10243B00E140089001D2E0640260469001D2E012C4
:0E244B00035E0003E0245924672481248C24BE
:102459009001D2E004F09001CFE0F5C280799001BB
:10246900DDE0A2E25007D2E4F0D2C5806A9001D241
:10247900E004F09001D080E19001D2E004F09001F5
:10248900D180D69001DDE0C2E0F0E49001D2F0D233
:10249900C48044E49001D2F0D2C480CD9001D2E04E
:1024A90012035E0101E024B424CC24E5C29001D0DA
:1024B900F09001D2E004F09001DDE0A2E1500AD2EF
:1024C900C18014E5C29001D1F0C2C1E49001D2F0FB
:1024D9009001DDE0C2E0F0C2C0D0F00223E0C0E02C
:1024E900C0D0C082C083D2909001DBE0D2E4F00278
:1024F90023E0C0E0C0D0EAC0E0C082C083900A21D6
:10250900E0FA74012AF0EAC39405405C75A60075E7
:10251900A0FFC296C2839001DEA2A5E092E0F0A2DC
:10252900A0E092E1F0A2A6E092E2F0A2A7E092E395
:10253900F0A2A2E092E4F0A2A1E092E5F0A2A3E069
:1025490092E6F0A2A4E092E7F0E064FF6013900144
:10255900DFE0A2E4400BE0D2E3F09001DBE0C2E36C
:10256900F0D296E4900A21F0C2CFD083D082D0E095
:10257900FA0223E4C2AD9001DFE0D2E4F074FF90E7
:1025890001DEF074029008F2F012173D7418900100
:10259900D0F074409001D1F074029001CFF0900115
:1025A900DFE0D2E2F09001DDE0C2E4F0D2E1F090A8
:1025B90001DFE0C2E1F012216AE0D2E2F01217D99C
:1025C90075A6FF7A537B74121C1A9001E37437F0D5
:1025D900A374FFF09001E57453F0A37474F07C3791
:1025E9007DFF7A237B00795A121D3B7582F375832F
:1025F900087E1E7F008012EEFAEFFB7919121C7417
:10260900EE240AFEEF3400FFA3E0FAFC743F6A707F
:10261900E6D2AD9001DEE064FF60F89001DFE0C230
:10262900E4F0C2AD121DDC121F8B9001DBE0D2E594
:10263900F0E0D2E3800EC296D2961226FDE0C2E304
:05264900F0E0D2E0F01A
:10264E00E0A2E54052E0A2E040FBE0A2E340E2E07F
:10265E00A2E1501F12207B9009747414F0A3E4F0D1
:10266E009001B27414F0A3E4F0D2999001DBE0C2B1
:10267E00E180C8E0A2E250C89001DDE0C2E4F012B1
:10268E00216A7401900978F09001DBE0C2E280AB20
:10269E0012207BE0C2E1F09001DBE0A2E5504F801A
:1026AE0005C2AD1228C6D2ADE0A2E340F4E0A2E12D
:1026BE0040DEE0A2E2501C9001DDE0C2E4F0122107
:1026CE006A7401900978F09001DBE0C2E2F0E0D28A
:1026DE00E380C39001DFE0A2E350BCC2AD122BD366
:1026EE00E0C2E3F09001DBE0A2E240AB80E022C06A
:1026FE0082C083D2A8C2909001DBE0A2E450F8E041
:10270E00C2E4F0C2A8D2909001D5E06004640270D9
:10271E00339001D3E4F0A3F0D297C297D2979001F1
:10272E00D3E02401F0A3E03400F09001D3C3E09491
:10273E00FFA3E0940140E1D2979001B2E4F0A374BC
:10274E0002F0D2999001B9E064016005E064027074
:10275E00089001DBE0A2E650F89001D5E06401603C
:10276E0005E0640270319001D3E4F0A3F0D295C27B
:10277E0095D2959001D3E02401F0A3E03400F090BF
:10278E0001D3C3E094FFA3E0940140E19001B2E4D1
:10279E00F0A37402F0D299C296D2960221C974F5B2
:1027AE001202C6750B00E49008F1F075A60075A034
:1027BE00FF780979057AFD7B067C10C297E5A02487
:1027CE0039F582E43404F583E49388828983F0D268
:1027DE0097C295E5A02439F582E43404F583E49399
:1027EE008A828B83F0D295A3AA82AB838882898357
:1027FE00A3A882A9831CEC70C2750A08781179050A
:04280E007A057B07C5
:10281200C297E82408FCE93400FDE5A02439F582DA
:10282200E43404F583E4938C828D83F0D297C295CD
:10283200EA2408FEEB3400FFE5A02439F582E434F3
:1028420004F583E4938E828F83F0D295E50B705169
:102852009008F2E0702788828983E0FEC3943D40AD
:1028620040EEC39444503A8C828D83E0FCEEC39CCC
:10287200502FE50A9008F1F0750B01802464017075
:10288200208A828B83E0FCC3943D4015ECC39444C0
:10289200500FECC0E08E828F83E0FCD0E0C39C40FE
:1028A200D1050A8A828B83A3AA82AB838882898319
:1028B200A3A882A983E50AC3945C50030228127F6D
:1028C2000402032674F11202C674FA12028CD2A810
:1028D200C2909001DBE0A2E450F8E0C2E4F0C2A8AA
:1028E2001227AC9008F2E06402700874019008F1BB
:1028F200F080099008F1E07003022BC77E007F0090
:1029020074041202BC746DF0A37405F07402120216
:10291200BC7461F0A37407F0750CE9750D017508BC
:10292200797509039008F1E0F82409FAE43405FB0B
:10293200851082851183EAF0A3EBF0E824FDF50E01
:10294200E43406F50F75A60075A0FFC297E5A02432
:1029520039F582E43404F583E493C0E0740412028E
:10296200BCE0F8A3E0F5838882D0E0F0D297C2956C
:10297200E5A02439F582E43404F583E493C0E074DD
:10298200021202BCE0F8A3E0F5838882D0E0F0D224
:102992009575A6FF850C82850D83E0FC74786C60CA
:1029A2000874C86E7001EF700B9001E774EFF0A32A
:1029B200747B8052EC75F00584E5F07011EEF8EF4F
:1029C200F97A197B00120210EA7001EB60DB8C0AC3
:1029D2007405250AF8E43400F97A197B001202081A
:1029E200EA7001EB7011EEF8EFF97A057B00120242
:1029F20010EA7001EB60B29001E5E0F8A3E0F99013
:072A020001E7E8F0A3E9F091
:102A0900EEFAEFFBECF9121BC69001E7E0FAA3E03E
:102A1900D283F5A0C280D280EAF5A0C280D280C25A
:102A290083850882850983E0FC74786C600874C822
:102A39006E7001EF700B9001E774EFF0A3747B8067
:102A490052EC75F00584E5F07011EEF8EFF97A199A
:102A59007B00120210EA7001EB60DB8C0A74052519
:102A69000AF8E43400F97A197B00120208EA7001C5
:102A7900EB7011EEF8EFF97A057B00120210EA709B
:102A890001EB60B29001E5E0F8A3E0F99001E7E815
:102A9900F0A3E9F0EEFAEFFBECF9121BC69001E79F
:102AA900E0FAA3E0D283F5A0C280D280EAF5A0C201
:102AB90080D280C2839001E774E6F0A374FFF085A9
:102AC9001082851183E0F8A3E0F5838882E0246E03
:102AD900F50AEEFAEFFBA90A121BC69001E7E0FA24
:102AE900A3E0D283F5A0C280D280EAF5A0C280D249
:102AF90080C283850C82850D83E50AF09001E77415
:102B0900BFF0A3741DF0850E82850F83E0F50AEEF0
:102B1900FAEFFBA90A121BC69001E7E0FAA3E0D27B
:102B290083F5A0C280D280EAF5A0C280D280C28398
:102B3900850882850983E50AF0EE24010EEF340049
:102B4900FF850E82850F83A385820E85830F8510ED
:102B590082851183E02401F8A3E03400F98510820D
:102B6900851183E8F0A3E9F0850882850983A385A7
:102B79008208858309850C82850D83A385820C854E
:102B8900830D74021202BCE02401F8A3E03400F9B9
:102B990074021202BCE8F0A3E9F074041202BCE06A
:102BA9002401F8A3E03400F974041202BCE8F0A38C
:102BB900E9F0C3EE948FEF94015003022947C296BE
:102BC900D29674061202A2021DD7C082C083900158
:102BD900DEE0A2E7E492E044FEF4FA9001D6E02AAE
:102BE900F09001DEE0A2E6E492E044FEF4FA9001FE
:0F2BF900D6E0C39AF064FF705D7407F075A6FF15
:102C08009001E7E4F0A3F09001DCE0D2E0F07C8FE3
:102C18007D017A007B007900121EF57C8F7D017A98
:102C2800007B0079EF121EF59001E774FAF0A374A7
:102C380047F09001DCE0D2E0F07C647D007A047B10
:102C48000179EF121EF57A009001DEE0A2E450034C
:102C5800022EB30A022EB9E0C394084004E4F080BF
:102C680018E012035E0007BE2E812CAF2CF72C460D
:102C78002D8D2DDC2D502E052C75A6FF9001E7E437
:102C8800F0A3F09001DCE0D2E0F07C8F7D017A00C7
:102C98007B007900121EF57C8F7D017A007B00791C
:102CA800EF121EF5022EBE75A6FF9001E7E4F0A311
:102CB800F09001DCE0D2E0F07C8F7D017A007B00AF
:102CC8007900121EF57C8F7D017A007B0079EF1266
:102CD8001EF59001E774FAF0A37447F09001DCE068
:102CE800D2E0F07CA07D007A147B00790080B27578
:102CF800A6FF9001E7E4F0A3F09001DCE0D2E0F059
:102D08007C8F7D017A007B007900121EF57C8F7D17
:102D1800017A007B0079EF121EF59001E774FAF052
:102D2800A37447F09001DCE0D2E0F07C6E7D007A7D
:102D3800BE7B007900121EF5122EC1022EBE75A6AA
:102D4800FF9001E7E4F0A3F09001DCE0D2E0F07C32
:102D58008F7D017A007B007900121EF57C8F7D0142
:102D68007A007B0079EF121EF59001E774FAF0A360
:102D78007447F09001DCE0D2E0F07C507D007A36B8
:102D88007B01022CF375A6FF9001E7E4F0A3F09015
:102D980001DCE0D2E0F07C8F7D017A007B007900D5
:102DA800121EF57C8F7D017A007B0079EF121EF5EB
:102DB8009001E774FAF0A37447F09001DCE0D2E0E8
:102DC800F07C3C7D007A147B0079EF121EF51230FE
:102DD800F0022EBE75A6FF9001E7E4F0A3F0900183
:102DE800DCE0D2E0F07C8F7D017A007B0079001274
:0F2DF8001EF57C8F7D017A007B0079EF121EF5AE
:102E07009001E774FAF0A37447F09001DCE0D2E098
:102E1700F07C327D007A5A7B0079EF121EF5900123
:102E2700DBC0829001DEE0A2E4758301D082E092EC
:102E3700E7F09001DBC0829001DEE0A2E5B3758385
:102E470001D082E092E7F0806E75A6FF9001E7E47B
:102E5700F0A3F09001DCE0D2E0F07C8F7D017A00F6
:102E67007B007900121EF57C8F7D017A007B00794B
:102E7700EF121EF59001E774FAF0A37447F0900182
:102E8700DCE0D2E0F07C647D007A967B0079EF127B
:102E97001EF57A009001DEE0A2E440030A8006E016
:102EA700A2E540011AEA25EAF5EA800BE0A2E5402F
:102EB700011AEA25FCF5FC0221C974F71202C6744F
:102EC700FA12028C9001DEE0A2E4406A9001DFE092
:102ED700A2E09001D95025E02401F0A3E03400F0EE
:102EE7009001D9C3E0941CA3E09400A2D265D0332B
:102EF700403C9001D9741BF0A3E48031C3E09418DF
:102F0700A3E09400A2D265D0339001D9E040102409
:102F170001F0A3E03400F09001DFE0D2E0800E245E
:102F270001F0A3E03400F09001DFE0C2E0F090018F
:102F3700DFE0C2E18031E0A2E550030230E8900112
:102F4700D9E024FFF0F8A3E034FFF0F9C3E89401D7
:102F5700E99400A2D265D03350D49001D9E4F0A30C
:102F6700F09001DFE0D2E1F0E0A2E1501B7418908D
:102F770001D7F074409001D8F074029001CFF0901F
:102F870001DFE0D2E2023031E0A2E0504C9001D9FB
:102F9700E0F508A3E0F5097808120394180003DCAC
:102FA7002FB02FC32FC72FD02F74189001D7F0E45D
:102FB7009001D8F09001DFE0C2E080187418800B10
:102FC70074199001D7F0E4800874199001D7F07450
:102FD700809001D8F07402804EE0A2E25004741889
:022FE70080E088
:102FE9009001D9E0F8A3E0F9E8C333F8E933F9E847
:102FF90024E9F582E93416F583E493C0E07401937A
:10300900F583D082AA82AB838A088B097402780877
:10301900120269E5089001D7F0EAC4333354C0902D
:1030290001D8F074019001CFF0851082851183A831
:1030390082A9839001D9E0FAA3E0FBEA75F006A41E
:10304900FAACF075F006EBA42CFBEA2479FAEB3420
:1030590009FB7C028A828B83E088828983F08A82D9
:103069008B83A3E088828983A3F08A828B83A3A3BD
:10307900E088828983A3A3F0EA24030A0A0AEB34CD
:1030890000FBE82403080808E93400F91CEC70C4C3
:103099008510828511837EC87F008012EEFAEFFBCE
:1030A9007901121C74EE240AFEEF3400FFA3E0FA42
:1030B900FC743F6A70E69001E5E4F0A3F09001D753
:1030C900E09001D0F09001D8E09001D1F09001DBBF
:1030D900E0C2E3F0E0D2E2F09001DDE0D2E1F07489
:1030E900061202A202207674F81202C69001DEE0EE
:1030F900A2E040479008F2E060109001E374E6F026
:10310900A374FFF0E49008F2800A7402F09001E3DE
:1031190074FFF0A3F075826E7583097E1E7F00E04F
:10312900FAFC743F6A6063EEFAEFFB79E1121C74F2
:10313900EE240AFEEF3400FFA380E4E0A2E1404A56
:103149009008F2E0640160119001E374BFF0A37488
:103159001DF074019008F2800A7402F09001E37482
:10316900FFF0A3F075826E7583097E1E7F008012C1
:10317900EEFAEFFB79E1121C74EE240AFEEF34003B
:10318900FFA3E0FAFC743F6A70E69001E374FFF074
:05319900A3F0021C6F11
:00000001FF
